:0200000480007A
:10000000B72F0000938F0F8073900F3015A8130047
:100010000000130000001300000013000000130094
:100020000000130000001300000013000000130084
:100030000000130000001300000013000000010086
:10004000970200009382020C73905230814001416C
:100050008141014281420143814301448144014580
:100060008145014681460147814701488148014950
:100070008149014A814A014B814B014C814C014D20
:10008000814D014E814E014F814F971102009381A6
:10009000A1C5170502001305E54697950300938552
:1000A000257501461122170502001305E53A97054B
:1000B0000200938525430146C52817A503001305B3
:1000C000657397B503009385A57237B6ABAB13067E
:1000D000B6BAD92817B103001301C171EF60601BD4
:1000E000860293D21200F512638802008242110147
:1000F0006F00001073002030824211017300203025
:10010000711116C0F3222034E3CC02FC82421101AB
:10011000130141F806C20AC40EC612C816CA1ACC88
:100120001ECE22D026D22AD42ED632D836DA3ADCC7
:100130003EDEC2C0C6C2CAC4CEC6D2C8D6CADACC97
:10014000DECEE2D0E6D2EAD4EED6F2D8F6DAFADCA7
:10015000FEDE73252034F32510340A8601A07310C7
:10016000153492402241B2414242D2426243F243AC
:10017000025492542255B2554256D2566257F25703
:10018000064896482649B649464AD64A664BF64B33
:10019000065C965C265DB65D465ED65E665FF65F83
:1001A0001301C1077300203010C16374B50011053D
:1001B000E5BF828000000000000000000000000099
:1001C000000000000000000000000000000000002F
:1001D000000000000000000000000000000000001F
:1001E000000000000000000000000000000000000F
:1001F000197106C00AC20EC412C616C81ACA1ECC8D
:1002000022CE26D02AD22ED432D636D83ADA3EDCC6
:1002100042DEC6C0CAC2CEC4D2C6D6C8DACADECC96
:10022000E2CEE6D0EAD2EED4F2D6F6D8FADAFEDCA6
:100230009702020083A2422723A02200F322103457
:1002400096DEEF00002B170102000321E125024199
:10025000F65273901234B72200009382028873A082
:10026000023082403242C2425243E24372448254DC
:100270001255A2553256C2565257E2577258864806
:100280001649A649364AC64A564BE64B764C865C1A
:10029000165DA65D365EC65E565FE65F0961730059
:1002A0002030970202009382E22523A0120023A2AD
:1002B000220023A4320023A6420023A8520023AA2E
:1002C000620023AC720023AE820023A0920223A21C
:1002D000A20223A4B20223A6C20223A8D20223AA06
:1002E000E20223ACF20223AE020323A0120523A2F2
:1002F000220523A4320523A6420523A8520523AADA
:10030000620523AC720523AE820523A0920723A2C7
:10031000A20723A4B20723A6C20723A8D20723AAB1
:10032000E20723ACF207EF5060021701020003213D
:10033000A1170241F65273901234B7220000938243
:10034000028873A0023082403242C2425243E243EA
:10035000724482541255A2553256C2565257E25731
:10036000725886481649A649364AC64A564BE64B45
:10037000764C865C165DA65D365EC65E565FE65FB1
:10038000096173002030970202009382A21783A0B4
:10039000020003A1420083A1820003A2C20083A243
:1003A000020103A3420183A3820103A4C20183A427
:1003B000020203A5420283A5820203A6C20283A60B
:1003C000020303A7420383A7820303A8C20383A8EF
:1003D000020403A9420483A9820403AAC20483AAD3
:1003E000020503AB420583AB820503ACC20583ACB7
:1003F000020603AD420683AD820603AEC20683AE9B
:10040000020703AFC20983AF820782807370043092
:10041000197106C00AC20EC412C616C81ACA1ECC6A
:1004200022CE26D02AD22ED432D636D83ADA3EDCA4
:1004300042DEC6C0CAC2CEC4D2C6D6C8DACADECC74
:10044000E2CEE6D0EAD2EED4F2D6F6D8FADAFEDC84
:100450009702020083A2420523A0220086DEEF203D
:10046000100A17010200032121040241F652739081
:100470001234B72200009382028873A002308240B7
:100480003242C2425243E243724482541255A25550
:100490003256C2565257E257725886481649A649F4
:1004A000364AC64A564BE64B764C865C165DA65DD0
:1004B000365EC65E565FE65F09617300203073707A
:1004C000043001A07310453082807325403073F0F2
:1004D00043308280970700009387A7FE232EB5FE46
:1004E0002322C5FA232635F82320F5F8130505F84D
:1004F0008280411106C6EF409062EF10306601E540
:10050000B24041018280B24041016F20407F011121
:100510004EC6AA891305800326CA52C406CE22CC31
:100520004AC856C2AE84328AEF30D06B630B050CDA
:1005300097070200938747F39C432A84B5CBB5E025
:10054000130944004A8544D4231A0402232844038F
:1005500023203401692613058401512697070200E0
:10056000938747F0984348548947B384974000C81D
:1005700040D004CC6369A70293172500AA978A0785
:10058000170502001305C5FF3E95CA85A12E054536
:10059000F2406244D2444249B249224A924A056139
:1005A0008280854471BF9707020023ADA7EAE9B7AF
:1005B000170502001305C5FC9707020023A687EA6A
:1005C0002926170502001305E5FC0126970A0200FB
:1005D000938A8AFD5685D52C17090200130909FE56
:1005E0004A85E52417050200130585FEF92C9707B7
:1005F000020023AF57E79707020023A927E7A9D0F6
:100600004DB77D5571B7011126CA4AC8970402003B
:10061000938484E517090200130989E49C4022CCE5
:10062000032409004EC606CE2A9413854700AE89DE
:10063000F52C8C4083270900C0C16375F40297072D
:1006400002009387A7E2884391054D2C6385090238
:100650008C406244F240D24442494E85B249E105A1
:10066000056169AC97070200938787E0884391058D
:100670007124E39F09FCF2406244D2444249B249EA
:100680000561828079714AD04ECE06D622D426D218
:1006900052CC56CA5AC85EC617090200130949EE61
:1006A00083270905970902009389C9DBB9C37370D1
:1006B00004308327C905C04713058401852C736066
:1006C000043093044400268595245C5483A60900D5
:1006D000A685139527003E950A052A874A9563F754
:1006E000F61417070200232FF7D6ED2A83270905F2
:1006F000DDFFEF10703E97070200938727D69843DF
:10070000970A0200938ACAD583A70A00198D170792
:1007100002002323A7D4170A0200130A6AD5970BF5
:100720000200938BABD4170B0200130BEBD251CD0D
:1007300085077D15170702002324F7D2170702004B
:10074000232CA7D003270A0081EF83A60B001706EE
:100750000200232DE6D017070200232BD7D03687BF
:100760001443F1D658474047584063FAE700C1B7F1
:10077000D84783A70A004047584063E5E7047370F1
:10078000043093044400268555221C54130584012B
:1007900091C3692A736004305C5403A70900A685DD
:1007A000139527003E950A054A956376F7001707CB
:1007B00002002329F7CA3D2283270A0098434DFBF4
:1007C00083A70A0003250B0025F583A60900170758
:1007D00002002325F7C8939726003387D7000A071E
:1007E0004A97184335E385CA9387F6FF1397270086
:1007F0003E970A074A97184331E391CB9387E6FF68
:10080000139727003E970A074A97184305EB1707E7
:1008100002002329F7C4B250225492540259F249DB
:10082000624AD24A424BB24B456182803305E900AD
:10083000552883270905E39C07E665BDBE86170793
:1008400002002321F7C28A07B6978A073307F90007
:100850005443A1073E99DC425CC363852703C84724
:100860002254B2509707020023A0A7C09254025905
:10087000F249624AD24A424BB24B032305000C595B
:1008800045610283DC435CC3D9BF411106C626C261
:1008900022C45C45C0479304840126854128A6856F
:1008A000170502001305C5D2352897070200938764
:1008B000A7BB9C434854B240DC5722449244333592
:1008C000F5001345150041018280930785007D578F
:1008D0005CC118C55CC51CC9232005008280232883
:1008E000050082805C41DCC1984798C598474CC39D
:1008F0008CC788C91C4185071CC182809041FD5767
:10090000130785006314F60039A83E875C439443BF
:10091000E37DD6FEDCC18CC798C54CC388C91C4199
:1009200085071CC1828018495C43EDB758411445C6
:100930001C4914C71845544154C3D8436314A70035
:100940001845D8C32328050088437D1588C38280B5
:100950003041AE8701CE4C455841B2954CC563E459
:10096000E5000C414CC53E856F301040828041113E
:1009700022C406C62A8426C2EF2090313C44635B21
:10098000F0025C5085CB9304440209A83C44FD1757
:100990003CC43C446350F0025C5089CF2685EF2074
:1009A000A0776DD5EF2090173C44FD173CC43C4424
:1009B000E344F0FEFD573CC4EF20D02FEF20502D34
:1009C0007C40635BF0021C4885CB9304040109A8BA
:1009D0007C40FD177CC07C406350F0021C4889CFEE
:1009E0002685EF2060736DD5EF2050137C40FD17F6
:1009F0007CC07C40E344F0FEFD577CC02244B24002
:100A0000924441016F20102B29C5411122C426C2F6
:100A10002A8406C6AE84EF20B02734405C5C1840C0
:100A2000232C0402B387F6027D5670C018C430C46C
:100A3000B386D740BA9736975CC058C491EC1C482F
:100A40009DE3EF203027B240224492440545410106
:100A500082807370043001A013050401BD351305B5
:100A60004402A535F9BF13050401EF20E06A85476C
:100A7000E319F5FC613AF1B701E57370043001A0A8
:100A8000011126CA4AC84EC606CE22CCB2892E898A
:100A9000AA84A5C53305B50213055505EF3090149A
:100AA0002A8435C1930745051CC144DC2320240555
:100AB000EF20101E34405C5C18407D56B387F60270
:100AC000232C040270C018C430C413050401B3867B
:100AD000D740BA9736975CC058C4C53B130544024B
:100AE000ED33EF20301D230834052285F2406244A7
:100AF000D2444249B2490561828013054005EF3076
:100B0000700E2A8401E57370043001A000C071BF2B
:100B100001E57370043001A06375B5007370043093
:100B200001A0411122C409462E84814506C6A93779
:100B300011C500DDB240224441018280737004304F
:100B400001A05D7186C6A2C4A6C2CAC04EDE52DC38
:100B500056DA5AD85ED632C6630B051C6383051C71
:100B600089476399F600585D85476305F700737000
:100B7000043001A03689AE842A84EF20A07C11E5E0
:100B8000B24781C77370043001A0EF207010185C69
:100B90005C5C014B894BFD59130A0401930A440222
:100BA0006365F70C63087919B247638307246315FB
:100BB0000B002808EF206069EF20D00FEF10C07005
:100BC000EF20100D7C4063943701232204043C4441
:100BD0006394370123240404EF20D00D6C0028080F
:100BE000EF20C06863100520EF20900A185C5C5C61
:100BF000630CF70AEF20100CEF2090093C44634F80
:100C0000F00039A85685EF20205119C1EF2000715E
:100C10003C44FD173CC43C446354F0005C50FDF37D
:100C200023243405EF201009EF2090067C40634F09
:100C3000F00039A85285EF20204E19C1EF20006E38
:100C40007C40FD177CC07C406354F0001C48FDF3E1
:100C500023223405EF201006EF10100C054BEF2077
:100C60003003185C5C5CE37FF7F230406306060CEF
:100C7000631109140844A685EF30100F1C4434405A
:100C80005840B6971CC463EBE70A1C5C14405850EC
:100C9000850714C41CDC45CB13054402EF20C04774
:100CA00085476312F50AD1A8EF20D000B2455285DE
:100CB000EF204028EF20C07D3C44634FF00039A86E
:100CC0005685EF20604519C1EF2040653C44FD1773
:100CD0003CC43C446354F0005C50FDF323243405D1
:100CE000EF20407DEF20C07A7C40634FF00039A8B0
:100CF0005285EF20604219C1EF2040627C40FD1711
:100D00007CC07C406354F0001C48FDF32322340572
:100D1000EF20407AEF10500031F1EFF02FEF054B4C
:100D20003DBF3C41E38E07E27370043001A0737055
:100D3000043001A0304029E61C4085C71C5C585097
:100D400085071CDC31FBEF20E0760545B6402644E4
:100D500096440649F259625AD25A425BB25B6161CB
:100D600082804840EF20206A1C5C585023220400F7
:100D700085071CDCE31207F279D5EFF02FE9E1B724
:100D80004844A685EF30407E3C4058441440B307A9
:100D9000F0403E9758C4637CD7025840BA975CC471
:100DA00009475C506306E902185C050718DCC1DFDF
:100DB000E5B54844A685EF30207B3C4058441440BC
:100DC000B307F0403E9758C4E37CD7FCF9B75C50BA
:100DD000185C79DB185C7D1718DC185C050718DCDB
:100DE000BDD35DBD22856136EF1000730145B9BFEB
:100DF000EF20406C014599BF411126C2AA8413051A
:100E0000400522C406C6EF30E05D2A8415CD232CB0
:100E10000502FD577CC10547410558DC3CC423222F
:100E2000040023200400232404002326040023209C
:100E3000040423089404513C130544027934814688
:100E4000014681452285F5392285B24022449244EB
:100E5000410182800DC5411122C426C206C64AC086
:100E6000032945002A84EF20204D8144630CA9000A
:100E7000B240224426850249924441018280737027
:100E8000043001A05C448544FD175CC4F5F3814641
:100E90000146814522857531E1BF25C1B1C90111E6
:100EA00022CC26CA4AC852C406CE4EC68947B6844A
:100EB00032892E8A2A846399F600585D854763013A
:100EC000F7067370043001A0EFF02FE0185C5C5C53
:100ED000AA896367F70281444E85EFF0AFDEF240E6
:100EE000624426854249D244B249224A0561828041
:100EF0003C41D5D77370043001A07370043001A059
:100F0000304049E21C40DDCB1C5C7D5785071CDC72
:100F10003C446388E7083C44854485073CC46DBF76
:100F2000EFF0AFDA185C5C5CAA89636DF7023040C1
:100F300071DA4844D285EF3020633C405844144075
:100F4000B307F0403E9758C46375D7005840BA972E
:100F50005CC48947E39AF4FA1C5CDDD71C5CFD177E
:100F60001CDC5DB7304059DE4844D285EF30C05FAD
:100F70003C4058441440B307F0403E9758C4E367E0
:100F8000D7FCD9BFDDF40844D285EF30E05D1C44C6
:100F900034405840B6971CC4E3E8E7F61C401CC434
:100FA000A5B75C5085448DDB13054402EF20C016C5
:100FB00005D5E30309F22320990039BF4840EF200B
:100FC00080442322040089B731CD3C4181C773702E
:100FD000043001A01C41B1CB011122CC26CA2A84C5
:100FE0004AC84EC606CE2E89EFF02FCE185C5C5C48
:100FF000AA898144637DF7001C5C7D5785071CDC52
:101000003C446389E7023C44854485073CC44E85E3
:10101000EFF04FCBF240624426854249D244B249B8
:10102000056182807370043001A05C41D5D7737074
:10103000043001A05C5099E38544D1BF13054402FC
:10104000EF20800D75D9E30909FE85472320F900BB
:10105000E5B7397106DE22DC26DA4AD84ED652D4FC
:1010600056D232C66302051C638A051AB68AAE8957
:101070002A84EF20202D11E5B24781C77370043018
:1010800001A0EF20E0401C5C63920714B247638E1E
:10109000070A2808EF20601BFD5413094402130AB5
:1010A0000401EF202041EF102022EF20603E7C4021
:1010B00063949700232204043C4463949700232400
:1010C0000404EF20203F6C002808EF20201A63134F
:1010D0000518EF20E03B1C5CADCFEF20A03DEF20DA
:1010E000203B3C44634FF00039A84A85EF20C00202
:1010F00019C1EF20A0223C44FD173CC43C4463547A
:10110000F0005C50FDF324C4EF20C03AEF204038DB
:101110007C40634FF00039A85285EF10F07F19C171
:10112000EF20C01F7C40FD177CC07C406354F00062
:101130001C48FDF364C0EF20E037EF10E03DEF20E6
:1011400020351C5CC1E7B247A9FFEF20A03601455E
:1011500055A0EF2020361C40DDC7B2454A85EF1070
:10116000705DEF20E0323C44634FF00039A84A85BF
:10117000EF10907A19C1EF20601A3C44FD173CC46F
:101180003C446354F0005C50FDF324C4EF208032F3
:10119000EF2000307C40634FF00039A85285EF10FB
:1011A000B07719C1EF2080177C40FD177CC07C40D0
:1011B0006354F0001C48FDF364C0EF20A02FEF1033
:1011C000A03531C9EF20C02C1C5CB5DFCE8522854F
:1011D0004444EFF0EFF7639C0A041C5C1840FD17D1
:1011E0001CDC01E7EF20803148C01C48A1EFEF2054
:1011F000602C0545F2506254D2544259B259225AD9
:10120000925A21618280EF20A0284840EF2080156B
:10121000EF20402A99B7EFF06F9F6DB73C41E3870D
:1012200007E47370043001A07370043001A05C50B7
:1012300044C4D5DF13054402EF10106E4DD9EFF012
:10124000EF9C75B713050401EF10106D8547E3108F
:10125000F5FAF5B72285EFF08FF1EF10E02B01459D
:1012600051BF1DC9411122C44AC006C626C244410D
:101270002E892A84EF20400C6383A40281464A868B
:1012800081452285F93385476300F502B240224447
:1012900092440249410182807370043001A05C4491
:1012A000054585075CC4DDB75C4485075CC4F9BFB0
:1012B00015CDADC9011122CC26CA4AC84EC652C4AA
:1012C0002A8406CE3289AE89EFF02FA01C5C2A8AD0
:1012D000814485E35285EFF0EF9EF240624426851B
:1012E0004249D244B249224A056182807370043077
:1012F00001A0304001CE4C445C40B2954CC463E444
:10130000F5000C404CC44E85EF3000261C5C7D5728
:10131000FD171CDC7C40638CE7007C40854485071E
:101320007CC04DBF3C41D9D77370043001A01C482C
:1013300099E3854445B713050401EF10F05D75D9B5
:10134000E30909FE85472320F900E5B721C93C419F
:10135000A1CDA1CB011122CC26CA4AC852C42A84ED
:1013600006CE4EC62E8AEFF04F961C5C2A89814429
:1013700091CB8329C400D2852285EFF06FDD8544AF
:10138000232634014A85EFF0EF93F240624426852C
:101390004249D244B249224A0561828073700430C6
:1013A00001A07370043001A0EDDF7370043001A060
:1013B00001E57370043001A0411122C42A8406C6DD
:1013C000EF20000D005CEF20E00EB24022852244A9
:1013D0004101828001E57370043001A0411106C60D
:1013E00022C42A84EF20C00A1C5C405C1D8CEF20C4
:1013F000600C2285B24022444101828019C1085DFF
:1014000082807370043001A01DCD978703009387FD
:10141000673AD843630CE502D847630CE504D84B20
:101420006307E504D84F6302E504D853630DE50272
:10143000D8576308E502D85B6303E502D85F630E03
:10144000E5006F30400C7370043001A001470E07B7
:10145000BA9723A007006F30000B1D47CDBF194777
:10146000FDB71547EDB71147DDB70D47CDB70947B4
:10147000F9BF0547E9BF684582806CC58280034596
:101480000505828009C5085D1335150082807370DB
:10149000043001A019C51C5D485D1D8D1335150074
:1014A00082807370043001A0411122C426C24AC058
:1014B00006C62A842E89B28473700430EF10507DE2
:1014C000185C5C5C630BF704EF10D07E7360043033
:1014D00073700430185C5C5C0145636AF7007360EC
:1014E0000430B2402244924402494101828030409B
:1014F00029C20844CA85EF3020071C4434405840B4
:10150000B6971CC463E4E7001C401CC41C5C585024
:1015100085071CDC1DE70545D9B7EF10B0798DE8CC
:1015200073600430B24022449244024901454101B3
:1015300082801C40E1FF4840EF10F06C2322040041
:10154000F1B713054402EFF04FB471D56D5541BFAB
:10155000930504012685EFF00F8B736004307155FD
:1015600049B7411122C406C62A84737004301C5D39
:1015700089EB25E273600430B24022440145410109
:10158000828073600430737004301C5D014599E7FC
:1015900073600430B2402244410182802E87304083
:1015A0004C445C40B2954CC463E4F5000C404CC420
:1015B0001C5C3A85FD171CDCEF20107B1C4899E36E
:1015C0000545F9B713050401EFF02FAC75D96D553A
:1015D000C1B7930545023285EFF0EF8273600430A6
:1015E00071554DBF411126C206C622C4185D5C5D0F
:1015F000B2846368F700B2402244268592444101D8
:10160000828030412A8415CA0845EF20F0751C44B9
:1016100034405840B6971CC463E4E7001C401CC427
:101620001C5C85071CDCE1F85C50F1D71305440213
:10163000EFF0AFA5B334A0007DBF1C41F5F34841E6
:10164000EF10705C23220400E1BF1C5DA9C74111AB
:1016500006C622C426C25C45032805045841C29729
:101660005CC563E4E7001C415CC5145D2E87BE8544
:101670009387F6FF1CDDB2842A8442863A85EF20E8
:10168000B06E9C4099E31C4889EBB24022449244DE
:101690000545410182800145828013050401EFF078
:1016A000CF9E65D585479CC0CDB7978703009387AC
:1016B0006710984305C3984705C7984B05C7984FCF
:1016C00005C7985305C7985705C7985B15C7985F16
:1016D00015C3828001470E07BA978CC3C8C38280A6
:1016E0000547D5BF0947C5BF0D47F5B71147E5B752
:1016F0001547D5B71D47C5B71947F1BF97870300F1
:101700009387470BD8436308E502D847630BE5028C
:10171000D84B630AE502D84F6309E502D853630842
:10172000E502D8576307E502D85B6308E502D85F96
:101730006303A702828001470E07BA9723A0070020
:1017400082800547D5BF0947C5BF0D47F5B711478B
:10175000E5B71547D5B71D47C5B71947F1BF4111C3
:1017600022C426C24AC02A8406C6AE843289EF103B
:1017700030527840FD576314F700232204043844A4
:10178000FD576314F70023240404EF10B0521C5CCF
:1017900099E74A86A68513054402EF10B00CEF10B6
:1017A000304F3C44635BF0025C5085CB93044402B1
:1017B00009A83C44FD173CC43C446350F0025C5013
:1017C00089CF2685EF1050156DD5EF1030353C448C
:1017D000FD173CC43C44E344F0FEFD573CC4EF100D
:1017E000704DEF10F04A7C40635BF0021C4885CBE3
:1017F0009304040109A87C40FD177CC07C40635021
:10180000F0021C4889CF2685EF1010116DD5EF101E
:10181000F0307C40FD177CC07C40E344F0FEFD5777
:101820007CC02244B2409244024941016F1090486A
:1018300005C579714ECE52CC06D63E8A22D426D228
:101840004AD056CA5AC85EC662C4A547BA8963F868
:10185000E7007370043001A07370043001A0AA8AFD
:10186000AE843289B68B428B6309082213050006C9
:10187000EF2050372A84630D05200A0923286503C9
:101880004A869305500A5A85EF20105C03C704006E
:101890001C587119230AE40203C704003E99137906
:1018A000C9FF79C783C71400A30AF40283C71400D1
:1018B000E1C383C72400230BF40283C72400CDCBEC
:1018C00083C73400A30BF40283C73400D5C383C796
:1018D0004400230CF40283C74400D9CB83C75400CF
:1018E000A30CF40283C75400C1C783C76400230D4F
:1018F000F40283C76400ADCF83C77400A30DF40264
:1019000083C77400B5C783C78400230EF40283C75E
:101910008400B9CF83C79400A30EF40283C7940058
:10192000A1CB83C7A400230FF40283C7A400A9C3DB
:1019300083C7B400A30FF40283C7B40095CB83C759
:10194000C4002300F40483C7C4009DC383C7D4002C
:10195000A300F40483C7D40081CF83C7E40023012C
:10196000F40483C7E40089C783C7F400A301F40427
:10197000130B44005A85A3010404232634032328AF
:101980003405232A0404EFE09FF513058401EFE0FA
:101990001FF5A947B3873741232C040400C81CCC8A
:1019A00040D023220404232E04045E86D6854A8573
:1019B000EFE05FB208C063040A0023208A0073705E
:1019C000043017F90100130969AC8327090097F463
:1019D0000100938464AD91C798409C407C43850787
:1019E0007CC317F70100130727AB1C43850797F645
:1019F000010023A3F6AA9C40D5CB8327090017FA40
:101A00000100130A2ABE89EB9C40DC5763E6F9000B
:101A100097F7010023AA87A897F70100938707A6E5
:101A2000984397F601009386A6A65C549442050756
:101A300017F601002324E6A438C463F6F60017F76E
:101A400001002327F7A45147B387E702DA8533055E
:101A5000FA00EFE03FE98327090081C79C40FC437F
:101A6000BDE383270900054499C79C40DC5763F414
:101A70003701EFE0BF992285B250225492540259A7
:101A8000F249624AD24A424BB24B224C45618280B3
:101A90005A85EF2050277D54F9BF13152600EF20FB
:101AA00070142A8BE31405DC7D54F1B797F701001D
:101AB00023AC879E184385476301F70217FA01009C
:101AC000130A4AB291BF984094407C43FD177CC3EF
:101AD000FC42C1FB7360043069B7814A17FA010008
:101AE000130A4AB0514CA94B33858A03850A529593
:101AF000EFE0BFDDE39A7AFF97FB0100938B0BBB0E
:101B00005E85EFE09FDC97FA0100938A6ABB5685F9
:101B1000EFE0BFDB17F501001305C5BBEFE0FFDA0F
:101B200017F50100130545BCEFE03FDA17F501009A
:101B30001305C5BCEFE07FD997F7010023A4779781
:101B400097F7010023AE5795C1BD411122C406C6C7
:101B500026C24AC02A847370043097F4010093842B
:101B6000E4929C40F9E311E497F701009387C7934F
:101B70008043130944004A85EFE05FDB1C5489C7AA
:101B800013058401EFE09FDACA8517F501001305FC
:101B9000A5B5EFE03FD597F70100938727909843CD
:101BA00097F701009387878D9C43050797F60100FF
:101BB00023A6E68E9840850797F6010023A0F68CB1
:101BC00001CB97F701009387278E9843784349EF1D
:101BD0009C40B1C797F701009387078D9843630F27
:101BE000870873700430984039EB17F7010013072A
:101BF000678B14439442A5E27D5797F6010023AD0D
:101C0000E686984009CF9843784311CB9843944394
:101C10007C43FD177CC3FC4299E373600430B240FF
:101C20002244924402494101828097F70100938740
:101C3000A78798439C437C4385077CC32DB7944377
:101C40009843F8420507F8C217F701001307878584
:101C500014439442D5D2184358475847584397F6EF
:101C6000010023ABE68071BF984394437C43FD178A
:101C70007CC3FC42B1FF7360043099BF97E7010059
:101C80009387477F9C4381C77370043001A022442F
:101C9000B2409244024941016FE04FF741C517F746
:101CA00001001307678014438147638BA606411127
:101CB00006C622C426C27370043097E601009386DC
:101CC000E67C9C4291C710431C437C4285077CC242
:101CD0009C42AA84404981C71C43FC43B9E797E76B
:101CE00001009387277C9C43638B870497E701005F
:101CF0009387077B9C436384870497F7010093874E
:101D0000E79F6309F40297F701009387E79D63015A
:101D1000F4028547B240224492443E8541018280CC
:101D20003E8582807370043001A0EF40E04B45BFD8
:101D30009147CDB79C5493B717008907E1BF8947F6
:101D4000D1BF7370043097E70100938727749843DD
:101D500009EF15C59C43485581CB97E70100938750
:101D6000A7749843784315E3828017E701001307AF
:101D7000A77314431843F8420507F8C261FD17E73B
:101D80000100130767720843F1B7984394437C43FB
:101D9000FD177CC3FC42E9FB736004308280411173
:101DA00022C42A8406C6EFE04FF211E497E701004F
:101DB0009387876F80434054EFE0CFF0B240228595
:101DC000224441018280A54763F5B7007370043057
:101DD00001A0011122CC06CE26CA4AC84EC652C462
:101DE0002A847370043017E901001309296A8327D4
:101DF0000900D5EF79C43C486389F50817E701006D
:101E00001307876A63FCB7001443638D860C18437D
:101E10004457B3B4950093C4140029A00443818CA3
:101E200093B4140058546384E70A1C4C2CC863C64E
:101E30000700A947B385B7400CCC93172700BA9782
:101E4000584897E901009389E9798A07CE97631B7F
:101E5000F702130A44005285EFE05FAD17E7010077
:101E6000130707635C5418436376F70017E7010014
:101E70002320F7625147B387E702D2853385F90003
:101E8000EFE05FA699C0EFE06FD88327090081CB10
:101E900097E70100938747619C43FC439DEBF24029
:101EA0006244D2444249B249224A0561828097E79E
:101EB00001009387675F98439C437C4385077CC3FD
:101EC0001DF897E701009387275E80432DB74CD418
:101ED000A9BF6244F240D2444249B249224A056154
:101EE0006F40803081443DBF25C1011126CA97E46F
:101EF00001009384645B9C4006CE22CC4AC84EC647
:101F0000638DA7027370043017E9010013090958A3
:101F10008327090091C798409C407C4385077CC378
:101F2000584997E701009387677D6302F70283278B
:101F3000090081C79C40FC43A5EBF2406244D244B7
:101F40004249B249056182807370043001A01C557A
:101F500017E7010013070778E38BE7FCE9FB930918
:101F600045002A844E85EFE07F9C17E701001307A8
:101F700027525C5418436376F70017E701002329C2
:101F8000F7505147B387E70217E501001305856550
:101F9000CE853E95EFE01F959C405854DC57E36892
:101FA000F7F8EFE0AFC661B76244F240D24442496D
:101FB000B24905616F40402315CD011122CC26CADC
:101FC0004AC82A8406CE4EC6EFE02FD0584897E77D
:101FD00001009387A7722A8981446300F7024A852A
:101FE000EFE04FCEF240624426854249D244B249E6
:101FF000056182807370043001A01C5417E5010054
:102000001305456DE38DA7FCF9FB97E70100938766
:1020100067469C43A9EB97E701009387E7489C43F9
:10202000445493094400DC574E85B3B4F400EFE008
:10203000FF8F17E701001307A7455C54184393C4AB
:1020400014006376F70017E701002323F744514794
:10205000B387E70217E501001305C558CE853E9505
:10206000EFE05F88ADBF93058401EFE0BF8785BFD8
:102070000111056506CE22CC26CA4AC84EC652C4F6
:1020800056C25AC0EF200036630E051AAA84130503
:102090000006EF2020352A84630A051C0566930597
:1020A000500A04D92685EF20205A04588567F11775
:1020B000BE94B7474C4593879744130A44005CD8B5
:1020C0005285230C0402A3010404232604022328BE
:1020D0000404232A0404EFE09F8013058401EFE049
:1020E0001F80A947232C0404F19800C81CCC40D0C1
:1020F00023220404232E040401469715000093852F
:10210000E5B12685EFE00FBD08C07370043017E914
:1021100001001309A9378327090097E4010093847C
:10212000A43891C798409C407C4385077CC317E73F
:102130000100130767361C43850797E6010023ADAE
:10214000F6349C40C9C38327090097E901009389AD
:10215000694981EB9C40DC5789E797E7010023A59B
:10216000873497E7010093876731984397E601002A
:10217000938606325C549442050717E60100232F2C
:10218000E62E38C463F6F60017E701002322F73085
:10219000139527003E950A05D2854E95EFE08FF402
:1021A0008327090081C79C40FC43DDE783270900A2
:1021B00091C39C40EF10704985476305F50C59E1C8
:1021C0007370043001A097E7010023AF872C1843F8
:1021D000854797E901009389E940E314F7F8CE8A2F
:1021E00017EB0100130B8B4C5685D10AEFE0EFED96
:1021F000E31C5BFF17E501001305454BEFE0EFEC37
:1022000097EA0100938ACA4B5685EFE00FEC17E579
:1022100001001305254CEFE04FEB17E50100130516
:10222000A54CEFE08FEA17E501001305254DEFE01F
:10223000CFE997E7010023A7672797E7010023A1CC
:10224000572705B7F2406244D2444249B249224A74
:10225000924A024B05618280984094407C43FD176E
:102260007CC3FC42A1F77360043089B76244F2403A
:102270004249B249224A924A024B2685D24405611C
:102280006F20602873700430FD5717E70100232585
:10229000F71E624497E7010023AAA71EF240D2442A
:1022A0004249B249224A924A024B97E7010023A3CE
:1022B000071E05616FD0FFFE7370043097E70100C1
:1022C00023A6071C6FE02F8C17E701001307871A5E
:1022D0001C4385071CC382807370043097E701009C
:1022E0009387C71A984305E317E701001307871A76
:1022F00008439C4381CB97E701009387E71A9843F3
:10230000784301EF828017E701001307E7191443B0
:102310001843F8420507F8C2C1BF984394437C4371
:10232000FD177CC3FC42F9FF7360043082804111C9
:1023300006C622C4EFE06F9997E7010093878715DF
:102340008043EFE02F98B2402285224441018280F1
:1023500097E701009387471488438280797106D6F6
:1023600022D426D24AD04ECE52CC56CA5AC85EC6C5
:1023700097E70100938707109C43B1EF17E701002F
:10238000130747111C43850797E6010023A4F610A5
:10239000832A0700638F0A0697E701009387C70D1A
:1023A0009C43814463F1FA0897E9010093898923EA
:1023B00017EA0100130A4A0F83270A008546D857F7
:1023C00093172700BA978A07BE9983A7090063FF6E
:1023D000F600854421A897E701009387E70A9C430C
:1023E0008144850717E701002320F70A97E70100DA
:1023F000938747099C4391C38544B2502254268554
:1024000002599254F249624AD24A424BB24B456158
:10241000828017E401001304E4081C409C43DDC3E0
:102420007370043001A017E401001304A40797E9B6
:1024300001009389291B17EA0100130AEA0617EB2A
:102440000100130BEB041C409C43B5C31C40DC474C
:1024500003A9C70083274900930B49005E8563EEFB
:10246000FA04EFE0AFCC832789021305890199C3F1
:10247000EFE0CFCB8327C90203270B00DE8513953E
:1024800027003E950A054E956376F70017E7010091
:102490002320F700EFE00FC583270A000327C902B6
:1024A000DC57E362F7FA1C4085449C43C5F3FD57B3
:1024B00017E701002322F7FC01B717E70100232DDE
:1024C000F7FADDBD17E70100130787FD1C4018432D
:1024D00097E6010023A8E6FC17E701002322F7FC9A
:1024E00097E701009387C7F99C43850717E7010029
:1024F0002328F7F81C409C4399E7FD5717E7010094
:10250000232CF7F651BD1C40DC47DC47DC4317E7C2
:1025100001002323F7F649B597E70100938787F574
:10252000984301E77370043001A0011106CE22CC5C
:1025300026CA4AC84EC652C456C25AC07370043026
:1025400097E40100938484F4984061EB98437D17ED
:1025500097E6010023A0E6F29C43D9EB97E7010040
:10256000938787F39C43C9C797EA0100938A8A0738
:1025700017EA0100130ACAF117E901001309C9F2A9
:10258000854919A83385EA00EFE0CFB58327090014
:102590005854DC576379F70483A70A0FC1CF83A788
:1025A000CA0FC04713058401EFE04FB8130B440076
:1025B0005A85EFE0AFB75C5483260A00DA8513959D
:1025C00027003E950A052A875695E3FDF6FA17E798
:1025D0000100232FF7EAEFE0EFB0832709005854FA
:1025E000DC57E36BF7FA97E7010023AD37E96DB7E6
:1025F00001449C4081CB97E701009387E7EA9C4325
:10260000FC4395E72285F2406244D2444249B249F4
:10261000224A924A024B0561828017E701001307A4
:10262000A7E814431843F8420507F8C205B7EF308E
:10263000B03BC9BF17E40100130404E51C4095C377
:102640001C40054999CF193B09C597E7010023AB09
:1026500027E31C40FD1717E701002327F7E21C4082
:10266000FDF397E701009387E7E198438547E3117E
:10267000F7F8EFD0BFD90544ADBF11CD81E5737038
:10268000043001A017E701001307C7DE1C4399C7F8
:102690007370043001A07370043001A0411122C492
:1026A00006C614431841850617E601002324D6DC2C
:1026B00097E60100938606DE94423304B70000C11A
:1026C00063F7E602637FE40063FD860097E701009D
:1026D000938787DD88431105EFE04FA52285EF3012
:1026E000702A1D3D01C9B240224441018280E36F3E
:1026F000E4FCD9BF2244B24041016FD03FD111C99F
:1027000017E70100130707D71C4391C77370043004
:1027100001A06FD0BFCF411106C622C41843AA87BB
:10272000050797E6010023A7E6D497E60100938604
:10273000A6D717E701001307E7D5184388423304EB
:10274000F7001105EFE08F9E2285EF30B023E933CB
:1027500011E52244B24041016FD05FCBB240224428
:1027600041018280411122C406C697E70100938788
:1027700067D09C430144850717E70100232CF7CE5F
:1027800097E70100938747D19C4363E0F51217EE6A
:102790000100130EEEF097E201009382E2E30144A0
:1027A0000147854F1303500A21A0311E638DC20BD0
:1027B00083278EFFBA86F5DB8327CEFFDC43232EEB
:1027C000FEFE638AC70F03AFC700DC432A97814E22
:1027D000232EFEFE6385C70783A8C700938748039F
:1027E000232017015CC383A788042326F7011CC795
:1027F00083A7C8021CCB83A70805232C07005CCB4A
:1028000003A808038347080063906704C28785070D
:1028100083C60700B3850741E38B66FE8981C20545
:10282000C181231EB700850E1307070263061F032D
:102830008327CEFFDC43232EFEFEE39FC7F98327C9
:102840004E00232EFEFE49BF8145231EB700850E94
:1028500013070702E31E1FFD769413175400311E61
:10286000BA86E397C2F597E701009387A7C303AE43
:10287000070083270E00639D070E97E701009387EB
:1028800027C203AE070083270E006392071817EED6
:102890000100130E2ED583274E109DE383278E1142
:1028A0006395072019C223200600BD312285B2405E
:1028B00022444101828083274E00232EFEFE21B751
:1028C00083278E1017EF0100130F8FE2DC4317E709
:1028D0000100232DF7E06380E73383A2C700DC43C8
:1028E000AA96814E17E701002322F7E0914F1303C8
:1028F000500A6388E70783A8C7009387480323A08B
:102900001601DCC283A7880423A6F6019CC683A710
:10291000C8029CCA83A7080523AC0600DCCA03A82A
:102920000803834708006391672AC287850703C7A6
:102930000700B3850741E30B67FE93D72500C20765
:10294000C183239EF600850E9386060263861229B4
:1029500083278E10DC4317E701002329F7D8E39C77
:10296000E7F983270E1117E701002321F7D861B794
:1029700083274E00130F8E00D4432322DE0063888A
:10298000E629B307E500D84283A2C600814E232280
:10299000EE00894F1303500A6306EF068328C70031
:1029A0001387480323A01701D8C303A7880423A6CD
:1029B000F70198C703A7C80298CB03A7080523AC63
:1029C0000700D8CB03A80803034708006318671C57
:1029D0004287050783460700B3050741E38B66FE80
:1029E00013D7250042074183239EE700850E938776
:1029F0000702638D121B83264E00D8422322EE006D
:102A0000E31EEFF80327CE002322EE0041BF832709
:102A10004E00130F8E00DC432322FE006384E71F69
:102A200083A2C700DC43AA96814E2322FE00894F71
:102A30001303500A6306FF0683A8C7009387480361
:102A400023A01601DCC283A7880423A6F6019CC636
:102A500083A7C8029CCA83A7080523AC0600DCCA6A
:102A600003A808038347080063966710C287850799
:102A700003C70700B3850741E30B67FE93D7250023
:102A8000C207C183239EF600850E93860602638BE0
:102A9000120F83274E00DC432322FE00E31EFFF8C3
:102AA0008327CE002322FE0041BF8327CE1197EE5D
:102AB0000100938E2EC5DC4317E701002322F7C4E3
:102AC0006384D71383AFC700DC433307D5000143CA
:102AD00097E6010023A6F6C20D4F89429308500ADB
:102AE0006387D707C8479307450308C35CC33C45C2
:102AF0002326E7011CC75C551CCB1C5599C3232614
:102B000057003C49232C07005CCB0328050383476F
:102B1000080063951705C287850783C60700B3853C
:102B20000741E38B16FF93D72500C207C183231EFD
:102B3000F700050313070702638AAF028327CE114C
:102B4000DC4397E6010023ADF6BAE39DD7F983276E
:102B50004E1297E6010023A5F6BA69B78147231EF6
:102B6000F700050313070702E39AAFFC1A94E31C6E
:102B700006D225BB8147239EF600850E938606026A
:102B8000E39912F117EE0100130ECEA583274E1024
:102B9000769493165400E38307D01DB30147239E18
:102BA000E700850E93870702E39712E597E7010098
:102BB0009387078F03AE07007694931654008327FC
:102BC0000E00E38607CCA1B58147239EF600850E53
:102BD00093860602E39E12D783278E11769493166E
:102BE0005400E38107CCD1B583274E1217E70100CB
:102BF0002328F7B0C1BD83270E1117E70100232753
:102C0000F7AEE1B98327CE002322FE0011BD832653
:102C1000CE002322DE00B5B3797126D24AD04ECE43
:102C200052CC56CA5AC85EC606D622D497E90100CD
:102C30009389498417E901001309C99A17EA010029
:102C4000130ACA8497EA0100938A0A8697EB010067
:102C5000938B8B8497E4010093844484054B21A8D3
:102C600083A7090003244910850717E701002323E0
:102C7000F7805D3011E89C40E5F783270900E37C8D
:102C8000FBFEEFD0AFF8C5BF7370043083270A0096
:102C9000B9E383270911C04713054400EFD01FC9CA
:102CA00083A70B00FD1717D701002327F77E9C4051
:102CB000FD1717D701002323F77E83270A0089C752
:102CC00083A70A00FC4385E30858EF10D003228550
:102CD000EF1070034DB703A70A0083A70A007C43D7
:102CE00085077CC37DB703A70A0083A60A007C433F
:102CF000FD177CC3FC42E9FB73600430F1B797D742
:102D00000100938727779C43DDE3411106C697D7DF
:102D1000010023A9077617D701001307E7781C43A2
:102D2000B7A6A5A59386565A9C5B8C43639BD5009A
:102D3000D0436318B60094476395C600DC476388A8
:102D4000D70008430C4393854503EF20807397D643
:102D500001009386E673904217E701001307878806
:102D600011A89C42B9CB9C42FD1717D60100232124
:102D7000F672904293172600B2978A07BA979C433F
:102D8000EDD3904293172600B2978A07B305F70058
:102D9000D441A107BA97D442D4C16383F602DC467A
:102DA000B24017D701002321F77041018280854787
:102DB00017D701002328F76C82807370043001A0BC
:102DC000D1473306F602D442329754C3C9BF01112A
:102DD0004AC806CE22CC26CA4EC62A897370043051
:102DE00097D401009384846A9C4017D40100130493
:102DF000A46BD9E76314090003290400930949006F
:102E00004E85EFD0BFB28327890289C71305890198
:102E1000EFD0DFB1CE8517E501001305258EEFD089
:102E20007FAC9C4081C71C40FC43ADE31C40638BDE
:102E300027079C409DCF737004309C40C1EB97D70F
:102E40000100938727669843184325EBFD5717D752
:102E500001002323F7629C4089CF1C40FC4391CBA7
:102E6000184014407C43FD177CC3FC4299E3736017
:102E70000430F2406244D2444249B2490561828042
:102E800018401C407C4385077CC3ADB718401440F4
:102E90007C43FD177CC3FC42D1FB736004301C40B3
:102EA000E39927F99C40A1C397D701009387875CDA
:102EB0009C43ADCB7370043001A09C43DC47DC47DE
:102EC000DC4317D701002329F75A71B718401C407B
:102ED0007C4385077CC397D701009387A75C984301
:102EE00018432DD7D9BF97D701009387E75A17D733
:102EF00001001307276F9C4303278711631DF70009
:102F0000F240624497D7010023A0075AD2444249B5
:102F1000B249056182806244F240D2444249B249DA
:102F20000561F1BB6244F240D2444249B2490561B5
:102F30006FD0CFCD3DC9411126C297D401009384F3
:102F4000A4564AC02E898C4006C622C4E105EFD0A3
:102F5000FF9A88401105EFD07F9DFD57630AF90461
:102F600097D7010093870753804398409C434A9426
:102F700040C3636CF40497D701009387A75288433A
:102F80008C409105EFD09F9797D701009387C74E4C
:102F90009C436376F40097D7010023AF874CB2407F
:102FA000224492440249410182807370043001A09E
:102FB0008C402244B2409244024917D501001305C7
:102FC000E573910541016FD0FF9197D70100938779
:102FD000274D884322448C40B240924402499105D7
:102FE00041016FD0BF9111C997D7010093878748DE
:102FF0009C4399E77370043001A07370043001A002
:10300000411126C297D401009384044A9840AE87A8
:103010008C40B7060080D58F06C622C41CCFE105C0
:103020003284EFD03F8C88401105EFD03F90FD57A0
:10303000630EF40097D701009387C7458843B240D9
:1030400092442295224441016F30C0138C402244A7
:10305000B240924417D501001305456A910541011C
:103060006FD05F8825CD411126C297D4010093848B
:10307000A4434AC02E898C4006C622C4E10532848E
:10308000EFD05F8688401105EFD05F8A8547630ADD
:10309000F40497D701009387E73F804398409C430F
:1030A0004A9440C3636CF40497D701009387873F29
:1030B00088438C409105EFD07F8497D70100938798
:1030C000A73B9C436376F40097D7010023A6873A79
:1030D000B24022449244024941018280737004301C
:1030E00001A08C402244B2409244024917D501000D
:1030F0001305C560910541016FD0CFFE97D7010040
:103100009387073A884322448C40B2409244024954
:10311000910541016FD08FFE411106C622C426C21F
:103120005C45C04735CC930484012685EFD01F80D1
:1031300097D70100938707349C43B5E79304440075
:103140002685EFD0AFFE97D7010093876734585498
:103150009C4363F6E70097D7010023ABE732931750
:103160002700BA978A0717D501001305A547A6853A
:103170003E95EFD02FF797D701009387E7329C4316
:1031800058540145DC5763F8E700854717D701001D
:10319000232AF72E0545B240224492444101828001
:1031A0007370043001A0A68517D501001305855260
:1031B000EFD04FF3C9B797D701009387A72B9C4354
:1031C00081E77370043001A0411106C622C426C2F3
:1031D000B70700804045CD8F1CC12DC4EFD00FF53F
:1031E000930444002685EFD06FF497D701009387AE
:1031F000272A58549C4363F6E70097D7010023A978
:10320000E72893172700BA978A0717D501001305F7
:10321000653D3E95A685EFD0EFEC97D701009387EB
:10322000A7289C4358540145DC5763F8E7008547BD
:1032300017D701002328F7240545B24022449244C1
:10324000410182807370043001A011CD97D7010035
:1032500093870723984397D701009387A7239C431D
:1032600018C15CC182807370043001A055C1D1CDFA
:10327000411106C622C42A877370043097D8010012
:103280009388C82083A7080091CB97D70100938724
:10329000A72194439C43FC428507FCC217D301003D
:1032A0001303431F9C4103260300FD560144638F13
:1032B000D70217DE0100130EAE1C03250E000328F3
:1032C000070054436305A80005446371D602330820
:1032D000D6400544637CF80003250E00918F032639
:1032E0000300B6979CC108C350C3014483A70800DC
:1032F00081CB97D701009387271B9C43FC4381EF29
:103300002285B2402244410182807370043001A0C2
:103310007370043001A0EF20306DDDB7854717D7FB
:1033200001002321F716828019C16845828001457A
:10333000828011C16CC5828097D701009387C71620
:103340008843828097D70100938747149C430545A3
:1033500089CB97D701009387E71188431335150070
:103360000605828031CD011126CA97D401009384CD
:10337000A4139C4006CE22CC4AC84EC65855DC57F2
:103380006379F7021C4D63C707009C40D457A947D7
:10339000958F1CCD93172700BA97584917D901006C
:1033A000130949248A07CA97630DF7009C40DC572C
:1033B0005CD5F2406244D2444249B2490561828000
:1033C0008280930945002A844E85EFD02FD69C40F9
:1033D00017D701001307C70B1843DC575CD463767B
:1033E000F70017D701002325F70A139527003E950C
:1033F00062440A05F240D244CE854A95B249424918
:1034000005616FD02FCE19CD411106C622C426C248
:1034100097D701009387470980436307A40073701F
:10342000043001A0014582807C4881E7737004303C
:1034300001A054543848FD177CC86383E60099C73F
:103440000145B240224492444101828093044400E9
:103450002685EFD0AFCD3C4817D7010013074703AF
:10346000144329471D8F5CD418CC63F6F60017D798
:103470000100232FF7005147B387E70217D501005A
:1034800013054516A6853E95EFD0CFC5054555BF1A
:103490007370043097D70100938747FF9C4391CB0B
:1034A00097D701009387470098439C437C43850747
:1034B0007CC3828097D70100938747FD9C438DC3CF
:1034C00097D70100938747FE9843784311CB9843E1
:1034D00094437C43FD177CC3FC4299E37360043042
:1034E000828097D70100938727FC904394439843A9
:1034F000A947D456084E958F1CCF828097D70100DC
:10350000938787FA984309C79443F84A0507F8CA8E
:103510008843828079714AD006D622D426D24ECEF4
:103520002A897370043097D40100938424F69C4058
:1035300017D40100130444F7BDE31C40BC4F89E7D6
:103540001C400547F8CFD1E19C4081C71C40FC439B
:10355000F1EB737004309C408DEF1C40A84F11C5F7
:10356000630409021C4023AC07041C4023AE07047B
:103570009C4081C71C40FC438DEBB25022549254B6
:103580000259F2494561828018403C4FFD173CCFFB
:10359000E9BF18401C407C4385077CC37DBF1840B1
:1035A0001C407C4385077CC349BF184014407C43C2
:1035B000FD177CC3FC42F1F373600430B250225417
:1035C00092540259F2494561828008402EC6110585
:1035D000EFD0CFB5B245FD576380F50697D7010010
:1035E000938747EB83A9070018409C43AE99232299
:1035F000370163ECF90497D701009387A7EA884362
:103600000C409105EFD08FAF97D701009387C7E6A5
:103610009C4363F6F90097D7010023AF37E5EFC06D
:10362000FFDE1DB7184014407C43FD177CC3FC42ED
:103630008DF37360043031BF0C4017D501001305C2
:10364000E50B9105EFD00FAAD9BF97D7010093875B
:1036500027E588430C409105EFD04FAAC9B779718F
:103660004AD04ECE06D622D426D252CC2E89B2894A
:103670007370043097D40100938444E19C4017D4C4
:103680000100130464E2F9EF18408947784F630C96
:10369000F7001C401345F5FFB84F798DA8CF1C40AB
:1036A0000547F8CFADE69C4081C71C40FC43F5E3DD
:1036B000737004309C40B1E7638609001C40BC4F26
:1036C00023A0F900184085470145784F630BF700A8
:1036D0001C401349F9FF0545B84F3379E90023AC85
:1036E00027051C4023AE07049C4081C71C40FC43B7
:1036F000C1E3B250225492540259F249624A4561E0
:10370000828018401C407C4385077CC375B7084005
:1037100036C61105EFD08FA1B246FD576385F60876
:1037200097D70100938707D703AA070018409C4347
:10373000369A232247016363FA0897D701009387DB
:1037400067D688430C409105EFD04F9B97D7010077
:10375000938787D29C436370FA0697D7010023AD05
:1037600047D191A818401C407C4385077CC329BFE2
:10377000184014407C43FD177CC3FC42BDFB7360C2
:103780000430B250225492540259F249624A4561BF
:103790008280184014407C43FD177CC3FC4289FBA7
:1037A0007360043031B70C4017D50100130505F5DF
:1037B0009105EFD02F93EFC07FC5F5B597D70100E6
:1037C000938707CE88430C409105EFD02F93E5B740
:1037D00051C1411106C622C426C24AC073700430CA
:1037E00097D40100938484CA9C40B9EB99C23C4DA4
:1037F0009CC2B2878946704D74CD2E872A84638619
:10380000D70663FCF6048D456387B7009145639541
:10381000B7006300D60C38CC8547630FF604054427
:103820009C4081CB97D70100938707C89C43FC43FA
:10383000A9E32285B2402244924402494101828098
:1038400097D70100938747C698439C437C438507DD
:103850007CC369BF7370043001A08546E39ED7FA2C
:103860003C4D33E7B70038CD45BF3C4D85073CCDD7
:1038700065B7EF20701775BF130944004A85EFD074
:10388000EF8A17D701001307A7C05C54184363766B
:10389000F70017D70100232DF7BE5147B387E70282
:1038A00017D50100130505D4CA853E95EFD08F8347
:1038B0001C5481C77370043001A097D7010093870F
:1038C000A7BE9C435854DC57E3FBE7F4EFC01FB49A
:1038D000B9B70144B1B739CD011122CC26CA4AC8C3
:1038E0004EC652C456C206CEBA89368AB2842E89D2
:1038F0002A84EFC09FBDAA8A63050A003C4C23209E
:10390000FA00784C89477CCC6389F40263F4970C05
:103910008D466387D40091466396D400630AF70A04
:10392000232C24058547631EF7061C5499CB73701E
:10393000043001A07370043001A03C4C85073CCCDE
:10394000D5B797D701009387E7B29C43ADEB9304BB
:1039500044002685EFC09FFD17D70100130747B32A
:103960005C5418436376F70017D701002322F7B29F
:103970005147B387E70217D501001305A5C6A685F1
:103980003E95EFC03FF697D701009387E7B19C4380
:103990005854DC5763F7E70063850900854723A087
:1039A000F90005445685EFC0FFB12285F24062441C
:1039B000D2444249B249224A924A05618280930523
:1039C000840117D501001305E5D0EFC0BFF165BF35
:1039D0000144C9BF8547E397F4F43C4C33E9270120
:1039E000232C240581B74DC1011122CC26CA2A847B
:1039F0004AC806CE4EC6AE84EFC03FAD8947744C70
:103A00007CCC3C4C05472A8985073CCC6395E6066F
:103A10001C5481C77370043001A097D701009387AD
:103A200067A59C43ADE7930944004E85EFC01FF0A6
:103A300017D701001307C7A55C5418436376F70036
:103A400017D701002326F7A45147B387E70217D5FC
:103A50000100130525B9CE853E95EFC0BFE897D785
:103A60000100938767A49C435854DC5763F5E70033
:103A700099C085479CC06244F240D244B2494A850D
:103A8000424905616FC01FA47370043001A0930503
:103A9000840117D501001305E5C3EFC0BFE4C1B72A
:103AA000AA8729C57370043017D701001307079E32
:103AB00014439DE2F04F894601456315D60023AEBD
:103AC000070405451C4381CB97D701009387C79D09
:103AD0009843784315E3828097D601009386C69C6D
:103AE000904294427442850674C2E9B797D70100A8
:103AF0009387879B9C437DB7984394437C43FD17F2
:103B00007CC3FC42E9FB7360043082805D71A6C215
:103B1000CAC052DC56DA5AD85ED686C6A2C44EDE79
:103B200062D466D26AD017D901001309E99817DB6D
:103B30000100130BAB9797D401009384649797DA35
:103B40000100938A2A97054AA54B832709009843C9
:103B500063010712DC4783A90700EFE0EFF6EFE00F
:103B6000AFF783270B002A8C6362F50A97D7010011
:103B700023AEA79201466370351B8840B385894107
:103B8000EFD0FFBDEFE05F996301051288408146E9
:103B900001462C00EFD0EFCB4DD9A247E3C807FE7A
:103BA000C24983A7490189C713854900EFC01FD8BF
:103BB000EFE08FF283270B002A8C636DF508A24794
:103BC00017D701002324878FE3E2FBFCB317FA0029
:103BD00013F70721631A071613F7770C6318071EEC
:103BE00093F70702C5D74E85EF00F01145B7DC47C4
:103BF000C04783AC0700930944004E85EFC01FD334
:103C00005C50228582975C4C6384470B83270900B4
:103C1000984371FF03A70A0097D6010023A886895D
:103C200097D6010023A8F68897D7010023A6E78836
:103C3000EFE09F8EA1BFDC47C04703AD0700930CA8
:103C400044006685EFC09FCE5C50228582975C4C15
:103C50006386470983270900984371FF03A70A0079
:103C600097D6010023A8F68497D7010023A6E784FE
:103C7000B9B7EFE06FE5EFE02FE683270B002A8C62
:103C8000E366F5F883A70A00884081499043B3852D
:103C9000894117D70100232B878113361600EFD0F7
:103CA0001FACEFE07F87E31305EEEFC02FF6F9BD01
:103CB0001C4CCE85E69763E9FC049C4089CF02CA80
:103CC00066CC22CEEFF00FE88840814601464C08D2
:103CD000EFC03FE705FD7370043001A01C4CE68582
:103CE000EA97636CFD049C4089CF02CA6ACC22CE5D
:103CF000EFF04FE58840814601464C08EFC07FE475
:103D000031F97370043001A0032509005CC000C8BC
:103D1000EFC0DFBEE5BDEFE03F8083270900DC4751
:103D2000C047930C44006685EFC05FC05C4C638F56
:103D300047035C502285829791BD032509005CC032
:103D400000C8EFC0BFBB39B7B24723ACF900A5CF5D
:103D5000E29723A2F90023A8390193854900636FF4
:103D6000FC0403A50A00EFC07FB90DB51C4C00C8C8
:103D70003387F90058C0636DEC02330C3C41636338
:103D8000FC029C4089CF02CA4ECC22CEEFF08FDBE2
:103D90008840814601464C08EFC0BFDA59F973707C
:103DA000043001A003A50A00E685EFC03FB551B776
:103DB00003250900E685EFC07FB4A5BF03250900F0
:103DC000EFC0DFB3E1B37370043001A0B24783A644
:103DD000890123A839013387D70023A2E90063644E
:103DE000EC04B307FC4063EBD70483A749024E857C
:103DF000829783A7C901E39B47D983A68901B2476C
:103E00009840B69711CF02CA3ECC4ECEEFF08FD37A
:103E10008840814601464C08EFC0BFD2E31805D662
:103E20007370043001A06374FC00E370F7FC032599
:103E3000090093854900EFC07FAC89BB03A50A0048
:103E400093854900EFC09FAB91B3411122C406C6D0
:103E500026C24AC017C4010013048465EFF04FE383
:103E60001C4095CBEFF00FE51C409DC381480148F5
:103E70008147094781461306004097C50100938595
:103E8000E553170500001305A5C8EFD07F9A39E95F
:103E90007370043001A017D90100130969874A859E
:103EA000EFC0BFA297D401009384C4872685EFC0DA
:103EB000DFA10146B145114597C7010023AE275F39
:103EC00097C7010023A8975EEFC01FBB17C701006B
:103ED0002320A75E11CD97C501009385A54DEFD096
:103EE000CFFC49B7B240224492440249410182804A
:103EF0007370043001A0A5C9797156CAAA8A130546
:103F0000C00222D426D24AD04ECE52CC06D65AC8AF
:103F10005EC63A89B689328AAE84E9212A8405C907
:103F2000EFF00FD797C70100938787589C439DCF29
:103F3000EFF04FD8130544002320540104CC232E66
:103F400044012320340323222403EFC05F992285F8
:103F5000B250225492540259F249624AD24A424B18
:103F6000B24B456182807370043001A097CB010091
:103F7000938B0B7A5E85EFC05F9517CB0100130B17
:103F80006B7A5A85EFC07F940146B145114597C7BA
:103F9000010023A3775397C7010023AD6751EFC0FA
:103FA000BFAD17C701002325A75001C997C5010060
:103FB00093854540EFD06FEFA5BF7370043001A02B
:103FC00039C5011122CC06CE26CA17C4010013043C
:103FD000244E832804002A88014563850802BA8498
:103FE0002EC2368732C442C6954663C5B602EFF08C
:103FF0006FB58947630BF5020840814601464C00C6
:10400000EFC03FB4F2406244D244056182807370D5
:10401000043001A04C0081463A864685EFC0FFE798
:10402000F2406244D244056182800840814626867F
:104030004C00EFC01FB1F9B719C1084182807370FD
:10404000043001A001E57370043001A0411106C6DF
:1040500022C42A84EFF0CFC348483334A000EFF0E5
:104060006FC52285B24022444101828001E5737010
:10407000043001A0411122C42A8406C6EFF04FC1CA
:104080000050EFF02FC3B2402285224441018280CC
:1040900001E57370043001A0411122C426C22E84B0
:1040A000AA8406C6EFF0CFBE80D02244B24092442C
:1040B00041016FF02FC04111714522C406C61D2673
:1040C0002A8411C5232005001105EFC01F80228519
:1040D000B24022444101828001CDB70700FFED8F3D
:1040E00081C77370043001A099E57370043001A09A
:1040F0007370043001A0011122CC4AC84EC652C4CC
:1041000056C206CE26CABA893689B28A2E842A8A2F
:10411000EFF04FA311E5638509007370043001A02F
:10412000EFE08F9A83240A00B377940063160902A4
:1041300095C763870A009347F4FFE58F2320FA00B1
:10414000EFE08FBDF240624426854249D244B24935
:10415000224A924A05618280E30DF4FCE38209FE63
:10416000B3355001E20563050900B7070004DD8D92
:104170004E86C18D13054A00EFE0FFE6EFE0CFB9B0
:1041800019E1EFC0AFA8EFF0CFB593176500AA898A
:1041900063D80700B7040001FD14B3F499005DB7BC
:1041A000EFF00FAF83290A00B3773401631E0900D3
:1041B00089CB63880A009347F4FFB3F737012320C4
:1041C000FA00EFF02FAFF9B7E31DF4FEDDB701C938
:1041D000B70700FFED8F99C77370043001A07370AB
:1041E000043001A0411122C42A8406C626C24AC056
:1041F0002E89EFF0EFA904409345F9FFB3F795003E
:104200001CC0EFF02FABB2402244268502499244F5
:1042100041018280411122C42A8406C6EFC0EFAA60
:104220000040EFC02FAAB240228522444101828083
:1042300009C9370700FFB3F7E50099C77370043069
:1042400001A07370043001A06F10D07BB70700FF8E
:10425000F18F81C77370043001A001E673700430E0
:1042600001A0011122CC4AC84EC652C406CE26CAAD
:104270003689AE892A8A3284EFF0CF8C21E163053A
:1042800009007370043001A0EFE00F8483240A005A
:10429000CE855285B3E49900613FB37794006307FC
:1042A000F40683240A00EFE02FA7F240624426853B
:1042B0004249D244B249224A05618280EFE0CF8070
:1042C00083240A00CE855285B3E434019537B3F7D1
:1042D0008400638D8702E30609FCB70500054A8662
:1042E000C18D13054A00EFE01FD0EFE0EFA219E106
:1042F000EFC0CF91EFF0EF9E93176500AA8463DFC4
:104300000700B7070001FD17FD8C45B783270A009A
:104310001344F4FFE18F2320FA0071B7EFF04F97B9
:1043200083240A00B3779400639787009347F4FFD0
:10433000E58F2320FA00EFF0EF97E1B7411122C497
:1043400006C62A8426C2EFD03FF85C4085C30848E1
:104350009304C4006316950015A0084863009502F5
:10436000B7050002EFE03FE55C40E5FB2285612AEE
:104370002244B240924441016FE00F9A73700430BE
:1043800001A009C9370700FFB3F7E50099C77370AB
:10439000043001A07370043001A06F10B06601C931
:1043A000B70700FFED8F99C77370043001A07370D9
:1043B000043001A0411122C426C206C62A84AE845C
:1043C000EFF00F8D184093C7F4FFF98F1CC0224403
:1043D000B240924441016FF0EF8D19C1084D8280C7
:1043E00001458280411122C406C62A84EFD0DFED48
:1043F00097C701009387870C9C43A1EBE56717C71C
:1044000001001307A733F11797C6010023AEE60A90
:1044100017C701002328F70A17C701002322F73224
:1044200097C701009387C70917C701002328F730F2
:10443000854717C70100232B070817C70100232151
:10444000070817C70100232BF70619E8EFE0CF8C08
:10445000EF10A00201442285B24022444101828033
:104460001305840093773500C1EFE5671307F5FF67
:10447000E917E3EDE7FC97C601009386E6049C424A
:1044800029A0984311C7BE86BA87D843E36BA7FE1D
:1044900017C701001307C702E38AE7FA98434146AA
:1044A0001384870098C2D843B306A7406378D60226
:1044B0003388A7002322D800C8C38325480097C6A5
:1044C00001009386660011A0BA8698425043E36DBE
:1044D000B6FE2320E80023A00601D84397C70100B9
:1044E000938787009C43998F17C70100232EF7FEFF
:1044F000EFE08F8231DC2285B2402244410182808C
:10450000719911059DB729C9411122C406C62A8493
:10451000EFD09FDB930584FF0326C4FF17C701007C
:10452000130787FA11A03E871C43D443E3EDC6FE70
:10453000232CF4FE0CC397C701009387E7FA984336
:104540008327C4FF2244B240BA9717C70100232D26
:10455000F7F841016FD05FFC828097C70100938715
:10456000A7F88843828082803367B5000D8BAA87C5
:104570001DE79308D6FFAA982A87AE8663711503B4
:1045800003A8060011079106232E07FFE36A17FF11
:104590009347F5FFC697F19B9107BE95AA972A9678
:1045A00063F3C70A9386450013884700B3B6D70064
:1045B00033B8050133E7F50093C616001348180019
:1045C0000D8BB3E6060113371700758F330EF640D7
:1045D0009386170029CF1337AE0031EB13532E000B
:1045E0002E88BE860147832808000507110823A0EE
:1045F00016019106E36967FE1377CEFFBA95BA9765
:104600006302EE0483C60500138717002380D700DA
:10461000637AC70283C6150013872700A380D700DB
:104620006372C70203C725002381E7008280B307B6
:10463000F640AE97850503C7F5FF8506238FE6FE96
:10464000E39AF5FE82808280B367C5008D8BB30844
:10465000C500E9C36371150FB307A0408D8B1387A5
:104660003700954693F5F50F130815003383A840DE
:104670007D166373D70015476363E60CD5CF23001F
:10468000B5000547638DE700A300B5000D4713088B
:1046900025006396E700130835002301B500139643
:1046A00085004D8E13970501518F3303F340939688
:1046B0008501D98E13562300AA97014794C3050795
:1046C0009107E36DC7FE1377C3FFB307E8006307E5
:1046D000E3062380B70013871700637C1703A380CA
:1046E000B70013872700637617032381B70013876A
:1046F000370063701703A381B70013874700637AFD
:1047000017012382B7001387570063741701A38230
:10471000B700828093F5F50F13978500D98D139715
:1047200005014D8FE37715FFAA87910723AEE7FEBA
:10473000E3ED17FF828082802A8895B78280AA875E
:1047400049BF834705002A8799C7050583470500A8
:10475000EDFF198D82800145828005058347F5FFB5
:10476000850503C7F5FF91C7E389E7FE3385E74079
:1047700082808147E5BFAA87850503C7F5FF8507C6
:10478000A38FE7FE75FB8280834605009307000236
:104790006397F600050583460500E38DF6FE9387D3
:1047A00056FD93F7D70F85C7AA87814585CE01456A
:1047B0008507138606FD1317250083C607003A9563
:1047C00006053295F5F699C13305A04082809385A0
:1047D00036FD8346150093B5150093071500E1FAE1
:1047E0000145D5B7014582809C412380A7009C41AB
:1047F00085079CC1828097C60100938666CD9C4246
:1048000017570300130707F413861700BA9723807E
:10481000A70097C5010023ADC5CAA9476308F500E5
:10482000930700046305F6000145828075DE3706B4
:1048300010F005078347F7FF2320F6F09C42FD1791
:1048400097C5010023A6F5C8EDF7014582804D719B
:104850002322911423202115232A51132324811369
:104860002326111423248114232E3113232C4113C6
:104870002328611323267113232291132320A113CC
:10488000232EB111AA842E8932C6130C5002A54AD8
:104890008347090063808703B9CB804011A0A1CB77
:1048A0002300F40080400509050480C08347090007
:1048B000E39787FF0346190093081900C686130D76
:1048C0000002FD597D5A0148130550059307D6FD96
:1048D00093F7F70F138916006363F52A17B70100E2
:1048E000130747728A07BA979C43BA978287832037
:1048F000C11403248114832441140329011483293E
:10490000C113032A8113832A4113032B0113832B21
:10491000C112032C8112832C4112032D0112832D0D
:10492000C11171618280A14C02C4854763D507150E
:10493000B2478040938B770093F68BFF03AB060062
:1049400083A94600938786003EC6668681465A85BF
:10495000CE85EF10E04D2AC8814763853723930D3C
:104960004101854B668681465A85CE85EF106016DB
:10497000814666862A8BAE89EF10804BA24723A022
:10498000AD0093861B00910D63843701B68BD9BFB0
:10499000E37E9BFF63DD4601A2872380A701804061
:1049A0007D1A930714009CC03E84E3C846FF93968B
:1049B0002B001C08BE9631A8938777052300F400CE
:1049C0008040FD1B93871B00050480C0F116E35156
:1049D000F0EC9C42E3E2FAFE93870703C5B79C40E4
:1049E0009306000332472380D7009C40930647007C
:1049F000C14C1386170090C013068007A380C70020
:104A0000804002C4BA87050480C003AB0700814917
:104A100036C625BFB24783AC0700938B470063843B
:104A20000C1C635F40199307D0026319FD1683C7FE
:104A30000C0085C363DC09189440850C7D1A238023
:104A4000F6008040050480C083C70C00E5F7635D75
:104A500040018040930700022300F40080407D1A4B
:104A6000050480C0E31A0AFE5EC61DB502C4854770
:104A7000A94CE3CF07EBB24780409386470071B75C
:104A800003C61600CA8699B59C409306500223803F
:104A9000D7008040050480C0E5BBC14C02C471B59D
:104AA000B24703C61600CA8683A9070091073EC60F
:104AB000E35E0AE04E8AFD5911BD03C61600130DD0
:104AC000D002CA8621B59347FAFFFD8703C61600B8
:104AD000337AFA00CA86DDBB03C61600130D000345
:104AE000CA86EDB383C51600930906FDCA8693876F
:104AF00005FD2E86E3EEFAFA93972900BE99850606
:104B00008609AE9983C50600938909FD938705FD43
:104B10002E86E3F3FAFE69BF32479C401443110727
:104B20003AC62380D7008040050480C095B38547EE
:104B300063D3070BB24793867700E19A9387860089
:104B40003EC683A946009C4263DC090A94401306D2
:104B5000D002B307F0402380C6008040B336F00097
:104B6000B3093041050480C03E8BB389D940A94CBC
:104B700002C4E1BB03C616000508CA8681BB9C407F
:104B8000468921B7E37D9BDD8547814B8546E3C59B
:104B900047E131BD97CC0100938CCC82CE856685F0
:104BA000EF001039330AAA40635C400180402300C3
:104BB000A40180407D1A050480C0E31A0AFE014A60
:104BC00083C70C00E38207EAE3C809E6FD197D57B5
:104BD000E394E9E6ADBDB247938647009C4336C6F1
:104BE00093D9F74195B7635640019307D002E31379
:104BF000FDFA97BC0100938CEC7C930780021DBDED
:104C00003E8BA94C02C4804089B34D71232E3113D1
:104C1000B70900409387F9FF2324811423229114BC
:104C2000232C4113232A5113232611142320211549
:104C30002328611323267113232481132322911324
:104C40002320A113232EB1112A8A2EC417C40100D8
:104C500013040488975A0300938ACAAE97B40100DC
:104C60009384C44F3EC6930550022945130800049F
:104C7000B70610F083470A006386B704C1C718401F
:104C8000050A13061700569797C8010023A2C88487
:104C90002300F7006382A706E31E06FD17570300F3
:104CA000130747AA05078347F7FF23A0F6F01C4028
:104CB000FD1717C60100232DF680EDF783470A0084
:104CC000E39EB7FA83461A0013051A002A87930B4E
:104CD00000027D5B7D5C014893055005A5489387E4
:104CE000D6FD93F7F70F130A170063E7F5348A0729
:104CF000A6979C43A697828717570300130787A49C
:104D000055F28DBF8320C1140324811483244114E0
:104D1000032901148329C113032A8113832A411310
:104D2000032B0113832BC112032C8112832C4112FC
:104D3000032D0112832DC11171618280A14C014D9F
:104D4000854763DB0719A2479D07E19B83AD0700F9
:104D500003AB4700138787003AC4668681466E8599
:104D6000DA85EF10E00C2AC863066D35130941019E
:104D70008549668681466E85DA85EF0090556686A0
:104D80008146AA8D2E8BEF10A00A2320A900850949
:104D90001109E3106DFFE3FE9DFD13060004B70645
:104DA00010F063D189031C4013871700D69797B57D
:104DB000010023AFE57023807701630CC7047D1CDD
:104DC000E3C389FFB2476800A548B386F9008A06A5
:104DD0001C08BE96294813030004370610F0E3842C
:104DE000A6E89C429305000363F4F8009305700560
:104DF0001840AE9793051700569717BE0100232958
:104E0000BE6C2300F7006380072B638C6526F116C8
:104E1000F9B7175703001307E79205078347F7FF12
:104E200023A0F6F01C40FD1797B5010023A2F56AF8
:104E3000EDF77D1C71B71C401306000413871700A3
:104E400097B5010023A6E568B386FA009305000331
:104E50002380B600630FC73C890797B6010023A9DA
:104E6000F6665697930680072300D700175703006E
:104E70001307478DB70610F0639EC70005078347E9
:104E8000F7FF23A0F6F01C40FD1717B60100232101
:104E9000F664EDF7A247C14C014D91072247014B43
:104EA000832D07003EC455BDA24783AC070013897C
:104EB0004700638E0C3A635480219307D002639EAF
:104EC000FB2E03C70C00BA856310072025AC85476D
:104ED000A94C014DE3C907E7A2479107C1B7A24713
:104EE00083461700528703AB070091073EC4E3587F
:104EF0000CDE5A8C7D5BE5B383461700930BD00222
:104F00005287F1BB9347FCFFFD8783461700337C34
:104F1000FC005287E9B383461700930B00035287C6
:104F20007DBB03461700138B06FD5287930706FDD2
:104F3000B286E3EEF8FA93172B00DA970507860797
:104F4000B29703460700138B07FD930706FDB28651
:104F5000E3F3F8FE69BFA2451C40294698419386B9
:104F60001700D69717B501002324D5562380E700F4
:104F7000138945006300C72A930700046387F6205E
:104F80004AC4D5B1854763DE0729A2471387770056
:104F9000619B930787003EC4032B47001C43635A61
:104FA0000B301840130600049306170097B5010054
:104FB00023A0D55256979305D0022300B7006387EC
:104FC000C62CB307F0403337F000330B6041BE8D81
:104FD000330BEB40A94C014D49B38346170005083C
:104FE0005287F5B9834617005287D5B91C409306FE
:104FF00000041387170017B60100232BE64CD69741
:10500000130650022380C700E31FD7C417470300CD
:1050100013074773B70610F005078347F7FF23A070
:10502000F6F01C40FD1717B601002323F64AEDF7F2
:105030001DB9C14C014D29B31C40930600042A8AB6
:105040001387170017B601002324E648D6971306E6
:1050500050022380C700E318D7C017470300130787
:10506000676EB70610F005078347F7FF23A0F6F039
:105070001C40FD1717B60100232CF644EDF72A8AD1
:10508000DDB6174703001307E76B05078347F7FFF4
:105090002320F6F01C40FD1797B5010023AAF54226
:1050A000EDF7F1162DBB174703001307A769F1FDB4
:1050B000F11635B3E3FC9DCB8549C5B1014C03C75F
:1050C0000C00BA85E30E07EAFD58294513080004D1
:1050D000B70610F063570B0A1C4013861700D697CB
:1050E00017B301002326C33E2380E7006384A5068F
:1050F00063040609850C03C70C007D1CBA8579FB87
:10510000E35080E91C409305000213060004B70633
:1051100010F021A07D1CE3050CE613871700D6973D
:105120002380B70017B501002324E53ABA87E313BB
:10513000C7FE174703001307E76005078347F7FF1C
:1051400023A0F6F01C40FD1717B501002322F53807
:10515000EDF7C9B7174703001307C75E41DE050720
:105160008347F7FF23A0F6F01C40FD1717B6010098
:105170002320F636EDF7BDBF174703001307875C02
:10518000F9BF7D1BE31A1BF5A5BF174703001307E3
:10519000675BB70610F005078347F7FF23A0F6F01B
:1051A0001C40FD1717B601002324F632EDF74AC460
:1051B0005DBC97BC0100938CEC20DA8566858D2B55
:1051C000330CAC40E35D80EF1C4013060004B706CF
:1051D00010F021A07D1CE3030CEE13871700D69777
:1051E0002380770197B5010023A4E52EBA87E31346
:1051F000C7FE174703001307E75405078347F7FF68
:1052000023A0F6F01C40FD1797B5010023A2F52C52
:10521000EDF7C9B7174703001307C752BDFA4AC4D1
:1052200099B4A247138747009C433AC413DBF74164
:10523000BDB3174703001307E750B70610F0050783
:105240008347F7FF23A0F6F01C40FD1717B60100B7
:105250002320F628EDF7854717B70100232AF72604
:105260009307800717470300230EF74C25B16356B9
:1052700080019307D002E39EFBF297BC0100938C60
:105280006C1413078002930580023DBD974603000E
:105290009386464B370610F0850603C7F6FF23209A
:1052A000E6F018407D1797B5010023A3E5226DF7BE
:1052B00009BBBE8DA94C014D4DB4B70710F023A01A
:1052C000A7F201A03971130341022ED29A8506CEAE
:1052D00032D436D63AD83EDA42DC46DE1AC6353209
:1052E000F2400145216182805D711303810322D464
:1052F0002AC632DC2A841A86680006D6BEC236DE8A
:10530000BAC0C2C4C6C61ACEEFF06FD4B24723806B
:1053100007003245B250018D225461618280B70787
:1053200010F083A647F403A607F403A747F4E31A93
:10533000D7FE8566938606FAB29633B6C600B305E5
:10534000E60023A4D7F423A6B7F48280B70710F0B1
:1053500003A747F403A607F483A647F4E31AD7FE8E
:105360008566938606FAB29633B6C60023A4D7F4B0
:10537000B305E60023A6B7F49307000873A04730EF
:105380008280411122C406C697B701009387C714D3
:1053900017B401001304041498431C401306F07C56
:1053A000930647069387470697B5010023A6D512B3
:1053B00097B5010023A0F5126346D600B2402244FF
:1053C000410182801307478997B7010023A6E710A0
:1053D000812E85476310F502184085679387F7761D
:1053E0000145E3DDE7FCEFF05FED2244B24041010F
:1053F0006FC09FEC17B50100130545FDEFF09FEC62
:105400000945EFF09FEB2244B24041016FC0DFEA53
:1054100017B50100130505FD6FF0DFEA17B50100B0
:105420001305C5FC6FF01FEA411122C426C206C64F
:10543000856417B401001304E4FB938784380100EA
:10544000FD17F5FF2285EFF0FFE7C5BF41AA411127
:1054500006C6F924054781476316E500B2403E853C
:105460004101828017B50100130545F6EFF09FE575
:10547000B24089473E85410182807370043001A0AB
:1054800082807370043001A0011126CA06CE22CC9E
:105490004AC84EC6835745031307901DAA84638BE1
:1054A000E70A6368F708D1CF1307801D639CE706FE
:1054B00013942500974903009389C92C33898900E7
:1054C000032509010146CA85EFC0AF89ED57630C7A
:1054D000F50E85476306F50017B701002324F70092
:1054E000B387890088530146CA85EFB0FFFBF157A7
:1054F0006304F508ED57630DF50A85476306F5006B
:1055000017B701002320F7FEB3878900884B7D562B
:10551000CA85EFC00F85F157E31AF5FA9307801D8E
:10552000239AF402F2406244D2444249B2490561EE
:1055300082801307E01E638CE7041307F01EE393D9
:10554000E7FE974903009389E923139425003389E3
:1055500089005DBF13942500974903009389892230
:10556000B38789008853338989000146CA85EFB023
:10557000BFF3F157E310F5F89307E01E239AF40206
:10558000F2406244D2444249B24905618280139498
:105590002500974903009389E91E33898900032573
:1055A00009020146CA85EFB03FF0ED57E317F5F465
:1055B0009307F01E239AF402F2406244D244424917
:1055C000B249056182809307901D239AF402F2404C
:1055D0006244D2444249B24905618280797122D441
:1055E00026D24AD04ECE06D602C6974403009384F4
:1055F000641B174903001309E919014497090000C6
:105600009389C9E8014691450545EFB0EFC688C0CA
:10561000014691450545EFB02FC62320A9008840DB
:1056200081466C000146EFB0CFD1228685454E857C
:10563000EFA0FFED0504914791041109E314F4FC78
:10564000B250225492540259F2494561828097B770
:1056500001009387E7E89C431307301F8507637CAD
:10566000F70A79714AD0174903001309A91322D404
:1056700026D24ECE52CC06D697B7010023A207E61B
:105680004A84974903009389E91217BA0100130A63
:10569000EAE48544084070002C0002C6EFB0FFFA2F
:1056A000630F950497B7010023AE97E21104E3134B
:1056B00034FF83270A00174403001304A40D97B98D
:1056C00001009389A9E1850717B701002328F7E0B6
:1056D000854408400146CE85EFB0DFF01104630633
:1056E000950097B7010023AF97DEE31489FEB2500F
:1056F000225492540259F249624A456182802247FB
:1057000083270A006306F70097B7010023AC97DCF4
:10571000B247C9FB61BF17B701002323F7DC8280C2
:1057200097B70100938707DC884313351500828003
:10573000AA95AA876385B70003C7070001E73385E9
:10574000A74082808507FDB7814863DA05003305ED
:10575000A040B337A000B305B0409D8DFD5863D97C
:1057600006003306C040B337C000B306D0409D8E5C
:1057700032883683AA872E87639F061C97B601005E
:10578000938646B363F1C50C416E6377C60B130E67
:10579000F00F6373CE002143335E6600F29603CEB2
:1057A00006001A9E130300023303C341630C030077
:1057B000B3956500335EC501331866003367BE00DC
:1057C000B3176500135E0801B355C703131508012D
:1057D000418193D607013376C703B305B50242066C
:1057E000D18E63F8B600C29663E5060163F3B60096
:1057F000C2968D8E33F7C603C207C183B3D6C603E4
:10580000B306D50213150701C98F63F8D700C297F5
:1058100063E5070163F3D700C297958F33D567001F
:105820008145638A0800B307A0403337F000B30511
:10583000B0403E85998D8280370E00014143E36D73
:10584000C6F5614391BF01E60548335868024167D8
:105850006373E8081307F00F63730701214333579D
:105860006800BA9603C606001A96130300023303B3
:10587000C34063190306B385054193560801131508
:105880000801418113D6070133F7D502B3D5D502FC
:105890004207518FB305B5026378B700429763653D
:1058A00007016373B7004297B305B74033F7D502DA
:1058B000C207C183B3D5D502B305B50213150701DD
:1058C000C98F63F8B700C29763E5070163F3B700B8
:1058D000C2978D8FA1B7370700014143E361E8F814
:1058E0006143B5BF3318680033DEC500935E08011D
:1058F0003356C500B31765003355DE03B395650015
:105900004D8E93150801C181935606013377DE034E
:105910003385A5024207558F6378A70042976365D8
:1059200007016373A7004297B306A74033F7D60376
:1059300042064182B3D6D6034207B386D502B36589
:10594000C70063F8D500C29563E5050163F3D50090
:10595000C295958D1DB7E3E6D5EC416863F5060564
:10596000930EF00F33B8DE000E0833DE060117B3D6
:105970000100130323947293834E0300130E00025D
:10598000C29E330EDE4163170E0263E4B600636904
:10599000C500B307C540958D3335F5003387A54065
:1059A0003E85BA85BDBD370300014148E3EF66FA85
:1059B000614865BF3357D601B396C601D98EB35738
:1059C000D50133D7D501B395C501CD8F93D5060148
:1059D0003373B702139F0601135F0F0113D807013A
:1059E0003316C6013315C5013357B7024203336876
:1059F0000301B30FEF023A83637CF8013698130377
:105A0000F7FF6367D8006375F8011303E7FF369863
:105A10003308F841B37FB8023358B802C20FB30558
:105A20000F03139F0701135F0F0133EFEF0142874D
:105A3000637CBF00369F1307F8FF6367DF00637561
:105A4000BF001307E8FF369F4203C16F3363E300D3
:105A50009387FFFF13580601330FBF40B375F30060
:105A600013530301F18F3387F502B307F302B385B4
:105A7000050333030303BE95135807012E98637380
:105A8000F8007E93C167FD17935508013378F8003D
:105A900042087D8F9A9542976366BF00631BBF00E3
:105AA0006379E5003306C7403337C700958D998D7C
:105AB00032873307E5403335E500B305BF40898DB4
:105AC000B397D5013357C70133E5E700B3D5C50117
:105AD00089BBAE87328836872A836396062097A8CB
:105AE00001009388287D63FEC50A41676374E60A56
:105AF0001307F00F3337C7000E07B356E600B6980A
:105B000083C60800369793060002998E99CAB39708
:105B1000D7003357E5003318D600B365F7003313C9
:105B2000D50013550801B3D7A50213160801418209
:105B30009356030133F7A502B305F6024207D98E47
:105B40003E8763FCB600C2961387F7FF63E7060142
:105B500063F5B6001387E7FFC2968D8EB3F7A602F2
:105B6000420313530301B3D6A602C20733E367000F
:105B7000B305D6023685637BB30042931385F6FFE7
:105B8000636603016374B3001385E6FF4207498F20
:105B900081454DA8B70600014147E360D6F661474D
:105BA000A9BF01E6854633D8C602C166637ED80820
:105BB0009306F00F63F306012147B356E800B69849
:105BC00083C60800BA9613070002158F49E7B3870A
:105BD00007418545135608019318080193D8080119
:105BE0009356030133F7C702B3D7C7024207D98ED2
:105BF0003385F8023E8763FCA600C2961387F7FF41
:105C000063E7060163F5A6001387E7FFC296898E56
:105C1000B3F7C602420313530301B3D6C602C20749
:105C200033E36700B388D8023685637B1301429360
:105C30001385F6FF63660301637413011385E6FFA2
:105C40004207498F3A858280B70600014147E366E3
:105C5000D8F661479DB73318E800B3D5D7003313A2
:105C6000E500B356D50013550801B397E70033F7A5
:105C7000A502B3E8F60093170801C18313D6080103
:105C8000B3D5A5024207518FB386B7022E86637C37
:105C9000D70042971386F5FF636707016375D70046
:105CA0001386E5FF4297B306D74033F7A602C20832
:105CB00093D80801B3D6A6024207B385D702B367CB
:105CC0001701368763FCB700C2971387F6FF63E7B7
:105CD000070163F5B7001387E6FFC2978D8F931511
:105CE0000601D98DC5BD63E2D514416763FEE602A6
:105CF0001308F00F3337D8000E0733D8E60097A506
:105D000001009385255BC29503C805009305000239
:105D10003A98B385054185E10547E3E5F6F2333569
:105D2000C5001347150039BFB70500014147E3E639
:105D3000B6FC6147D9B733570601B396B600D98E82
:105D400093DE060133D70701B378D703B397B700C3
:105D5000335805013363F80093970601C183135844
:105D600003013316B6003357D703C20833E80801DE
:105D7000338FE7023A8E637CE8013698130EF7FF03
:105D80006367D8006375E801130EE7FF36983308A0
:105D9000E841B378D8033358D803C208B38E070359
:105DA00093170301C183B3E7F800428763FCD7016F
:105DB000B6971307F8FF63E7D70063F5D70113071A
:105DC000E8FFB697420EB387D741C16E3367EE0046
:105DD0001388FEFF337307019358070133780601D8
:105DE0004182330E03033388080393560E013303B5
:105DF000C30242939A96B388C80263F30601F698E9
:105E000013D60601B29863E01703E39317D9C1676D
:105E1000FD17FD8EC206337EFE003315B500F296E7
:105E20008145E371D5E27D17A5B38145014719BDD1
:105E3000B2883687AA872E886398061C97A6010029
:105E40009386464763F8C50A4163637E6608130379
:105E5000F00F6373C30021473353E6009A9603CED5
:105E60000600130300023A9E3303C341630C030090
:105E7000B3956500335EC501B31866003368BE0094
:105E8000B317650013D608013377C80213950801CC
:105E9000418193D607013358C8024207D98E33088F
:105EA000050363F80601C69663E5160163F3060170
:105EB000C696B386064133F7C602C207C183B3D67E
:105EC000C602B306D50213150701C98F63F8D700C0
:105ED000C69763E5170163F3D700C697958F33D54F
:105EE000670081458280370300014147E36666F61B
:105EF00061479DB701E60546B3581603416663F353
:105F0000C8081306F00F63731601214733D6E80063
:105F1000B29603CE0600130300023A9E3303C34138
:105F200063190306B385154113D7080113950801BA
:105F3000418113D60701B3F6E502B3D5E502C206E7
:105F4000D18EB305B50263F8B600C69663E51601B7
:105F500063F3B600C696B385B640B3F6E502C20752
:105F6000C183B3D5E502B305B50213950601C98F08
:105F700063F8B700C69763E5170163F3B700C697E8
:105F80008D8FB1BF370600014147E3E1C8F8614793
:105F9000B5BFB398680033D7C501B3176500335E4A
:105FA000C50113D50801B376A702B3956500336E1A
:105FB000BE0093950801C18113560E013357A70205
:105FC000C206D18E3387E50263F8E600C69663E524
:105FD000160163F3E600C6963386E640B376A60262
:105FE000420E135E0E013356A602C2063386C50268
:105FF000B3E5C60163F8C500C69563E5150163F313
:10600000C500C695918D0DB7E3EED5EC416763F5FC
:10601000E604930EF00F33B7DE000E0733D3E6002D
:1060200097A80100938808299A9883CE0800130E38
:106030000002BA9E330EDE4163170E0263E4B6001F
:106040006369C500B307C540958D3335F5003388C6
:10605000A5403E85C28579B5B70800014147E3EF09
:1060600016FB614765BF3357D601B396C601D98E7B
:10607000B357D50133D7D501B395C501CD8F93D58E
:1060800006013373B702139F0601135F0F0193D804
:1060900007013316C6013315C5013357B702420352
:1060A000B36813013308EF023A8363FC0801B69822
:1060B0001303F7FF63E7D80063F508011303E7FF55
:1060C000B698B3880841B3FFB802B3D8B802C20F7C
:1060D000B3051F03139F0701135F0F0133EFEF0198
:1060E0004687637CBF00369F1387F8FF6367DF0036
:1060F0006375BF001387E8FF369F4203C1683363AF
:10610000E3009387F8FF13580601330FBF40B375C0
:10611000F30013530301F18F3387F502B307F30242
:10612000B385050333030303BE95135807012E9867
:106130006373F8004693C167FD17935508013378E0
:10614000F80042087D8F9A9542976366BF00631BF3
:10615000BF006379E5003306C7403337C700958D2C
:10616000998D32873307E5403335E500B305BF40ED
:10617000898DB397D5013357C70133E5E700B3D510
:10618000C5018DB397A7010093870732944317A7E2
:106190000100130727301843C8C2637BE50017A727
:1061A00001001307E72F08438C4391056FA00FF5FB
:1061B000411122C406C617A701001307A72E2A847F
:1061C00008438C439105EFA06FF397A701009387D5
:1061D000A72A9C436376F40097A7010023AE872883
:1061E000B24022444101828097A701009387C72BC8
:1061F000984394437C43FD177CC3FC4299E373604E
:1062000004308280011122CC26CA2A84AE844AC876
:106210004EC652C456C206CEEFC00F8B1C40032997
:106220000401B7090001B3E59700930AC4000CC04C
:106230008144FD19370A00021840638C2A030326A3
:1062400009004A85B3654701B376360193175600B6
:10625000758F0329490063C4070001E7F1BFE39D7F
:10626000E6FC9317760063D30700D58CEFC0BFF42C
:10627000E1B793C4F4FFF98C04C0EFC0EFA9084064
:10628000F2406244D2444249B249224A924A0561EC
:106290008280411106C622C4EFF04FB417F7FFFF0A
:1062A0001307670E814605469305400617A50100B2
:1062B0001305C514EFD03FC419C92A84EFC0CF819C
:1062C0002A860147814685452285EFD07FCFEFB0F2
:0C62D0003FDAB2402244014541018280C7
:02000004800278
:10000000804AFEFF7E4BFEFF884AFEFF7E4BFEFFCE
:100010007E4BFEFF7E4BFEFF7E4BFEFFA04AFEFFA7
:100020007E4BFEFF7E4BFEFFBA4AFEFFC64AFEFF36
:100030007E4BFEFFD84AFEFFE44AFEFFE44AFEFF85
:10004000E44AFEFFE44AFEFFE44AFEFFE44AFEFF04
:10005000E44AFEFFE44AFEFFE44AFEFF7E4BFEFF59
:100060007E4BFEFF7E4BFEFF7E4BFEFF7E4BFEFF78
:100070007E4BFEFF7E4BFEFF7E4BFEFF7E4BFEFF68
:100080007E4BFEFF7E4BFEFF7E4BFEFF7E4BFEFF58
:100090007E4BFEFF7E4BFEFF7E4BFEFF7E4BFEFF48
:1000A0007E4BFEFF7E4BFEFF7E4BFEFF7E4BFEFF38
:1000B0007E4BFEFF7E4BFEFF7E4BFEFF7E4BFEFF28
:1000C0007E4BFEFF7E4BFEFF7E4BFEFF7E4BFEFF18
:1000D0007E4BFEFF7E4BFEFF7E4BFEFF7E4BFEFF08
:1000E0007E4BFEFF7E4BFEFF7E4BFEFF7E4BFEFFF8
:1000F0007E4BFEFF7E4BFEFF7E4BFEFF7E4BFEFFE8
:10010000184BFEFF2E4BFEFF7E4BFEFF7E4BFEFF8D
:100110007E4BFEFF7E4BFEFF7E4BFEFF7E4BFEFFC7
:100120007E4BFEFF744BFEFF7E4BFEFF7E4BFEFFC1
:100130002649FEFFDE49FEFF7E4BFEFF7E4BFEFFA3
:10014000144AFEFF7E4BFEFF6C4AFEFF7E4BFEFF15
:100150007E4BFEFF9A4AFEFF8C4EFEFFE04EFEFFF6
:10016000944EFEFFE04EFEFFE04EFEFFE04EFEFF2F
:10017000E04EFEFF864DFEFFE04EFEFFE04EFEFF2E
:10018000A04DFEFFAC4DFEFFE04EFEFFBE4DFEFF5C
:10019000CA4DFEFFCA4DFEFFCA4DFEFFCA4DFEFF0F
:1001A000CA4DFEFFCA4DFEFFCA4DFEFFCA4DFEFFFF
:1001B000CA4DFEFFE04EFEFFE04EFEFFE04EFEFFAA
:1001C000E04EFEFFE04EFEFFE04EFEFFE04EFEFF83
:1001D000E04EFEFFE04EFEFFE04EFEFFE04EFEFF73
:1001E000E04EFEFFE04EFEFFE04EFEFFE04EFEFF63
:1001F000E04EFEFFE04EFEFFE04EFEFFE04EFEFF53
:10020000E04EFEFFE04EFEFFE04EFEFFE04EFEFF42
:10021000E04EFEFFE04EFEFFE04EFEFFE04EFEFF32
:10022000E04EFEFFE04EFEFFE04EFEFFE04EFEFF22
:10023000E04EFEFFE04EFEFFE04EFEFFE04EFEFF12
:10024000E04EFEFFE04EFEFFE04EFEFFE04EFEFF02
:10025000E04EFEFFE04EFEFFFE4DFEFF2C4EFEFF89
:10026000E04EFEFFE04EFEFFE04EFEFFE04EFEFFE2
:10027000E04EFEFFE04EFEFFE04EFEFF824EFEFF30
:10028000E04EFEFFE04EFEFFE44BFEFFDE4CFEFFC5
:10029000E04EFEFFE04EFEFF504DFEFFE04EFEFF43
:1002A000764DFEFFE04EFEFFE04EFEFFDA4EFEFF13
:1002B000000102020303030304040404040404040D
:1002C00005050505050505050505050505050505DE
:1002D00006060606060606060606060606060606BE
:1002E00006060606060606060606060606060606AE
:1002F000070707070707070707070707070707078E
:10030000070707070707070707070707070707077D
:10031000070707070707070707070707070707076D
:10032000070707070707070707070707070707075D
:10033000080808080808080808080808080808083D
:10034000080808080808080808080808080808082D
:10035000080808080808080808080808080808081D
:10036000080808080808080808080808080808080D
:1003700008080808080808080808080808080808FD
:1003800008080808080808080808080808080808ED
:1003900008080808080808080808080808080808DD
:1003A00008080808080808080808080808080808CD
:1003B000546D725100000000546D7220537663003A
:1003C000286E756C6C2900004572726F7220696E20
:1003D00020787878207461736B73200D0A00000018
:1003E0006D69616F750A00006D69616F75320A0091
:1003F00068756E6772790A00436865636B54696D4E
:040400006572000021
:100404001000000000000000017A5200017C01018C
:100414001B0D020010000000180000002853FEFF0E
:100424008A03000000000000100000002C000000FF
:100434009E56FEFF5E030000000000001000000056
:1004440040000000E859FEFF5403000000000000D3
:0804E400FC8F0100090000007B
:040000058000004037
:00000001FF
